:0300000002103AB1
:03000B000200A24E
:03002B000202CB03
:03005B0002041587
:030073000203EF96
:1000800002030406080C10182030406080040608A3
:100090000C10182030406080A0C005050D0502033B
:1000A0000302C2AFC0D0C0E020622C20680241B77A
:1000B0003066024177302F02E4730563C3740595FF
:1000C0002540F5956340F12069EE758A78E5257045
:1000D00003758A000202C485258AC262E525F47090
:1000E00002213E206802212B758B00D0E0D0D0C2C7
:1000F00092C291C290D2AF32C292C291C2907401A8
:10010000D5E0FDE53C1420E21520E10D207D02D272
:1001100093307D02D29502013BD29402013B207DB7
:1001200002D295307D02D29302013B758B00D0E064
:10013000D0D0C292C291C290D2AF32758B00D0E0C3
:10014000D0D0D2AF3241B7E525600A207D02D292ED
:10015000307D02D290C29141B7E5256002D2912054
:100160007D02C290307D02C29241B7E525600A202F
:100170007D02D290307D02D292207D02C292307DEB
:1001800002C29041B7207D02C295307D02C2932009
:100190007D02C293307D02C2957432D5E0FDE52523
:1001A000600A207D02D292307D02D290C29141B786
:1001B000207D02C295307D02C293C2947432D5E094
:1001C000FDE525600A207D02D292307D02D290C2E8
:1001D0009141B7C294207D02C295307D02C29374D2
:1001E00032D5E0FDE5256002D291207D02C290303B
:1001F0007D02C29241B7C294207D02C293307D023B
:10020000C2957432D5E0FDE5256002D291207D02D1
:10021000C290307D02C29241B7207D02C293307DF0
:1002200002C295C2947432D5E0FDE525600A207DB6
:1002300002D290307D02D292207D02C292307D02A5
:10024000C29041B7207D02C293307D02C295207DCD
:1002500002C295307D02C2937432D5E0FDE525607F
:100260000A207D02D290307D02D292207D02C2927D
:10027000307D02C29041B730723DE53C20E21A2049
:10028000E129207D02C295307D02C293207D02C209
:1002900093307D02C2950202B720E1E6207D02C2C2
:1002A00095307D02C293C2940202B7C294207D02AF
:1002B000C293307D02C295E525F4F58A758B0075F1
:1002C0006300D262D0E0D0D0D2AF32C2AFC2AD5361
:1002D000E6EFC0D0C0E0D2D3D2AFC2CEE5296007EE
:1002E0002074461529612978007900E580307E0167
:1002F000F430E70278FF53DACF207E0343DA203070
:100300007E0343DA10C2D8C271E580307E01F4303A
:10031000E70279FFC3E89970CE3061037529182090
:1003200074037529188859D270E52A6004152A616A
:100330003920740543DA01C2D82070026194A859AB
:10034000206102C270207431C3E894F0400374F05D
:10035000F8E8C4540F28F87984B703026179C3130D
:10036000C3138721200802C313200A06C3C898F8C4
:10037000617928F8500374FFF8C3E895625003E5EB
:1003800062F8882230690AC3E522955E4003855EE3
:1003900022852224A824C3E524955E4002A85E8815
:1003A00025C3E52594404002D26420CF0CD0E0D094
:1003B000D0C2D343E610D2AD32C2CF7801E5296076
:1003C000053074021529C3E55994014005755C0098
:1003D00061E3755D00756400E55C2401F55C500324
:1003E000755CFFD0E0D0D0C2D343E610D2AD32C0AE
:1003F000D0C0E0C2AF53917F53E67FC260759100D9
:10040000C3E49550F594E49551F595759104D0E0C9
:10041000D0D0D2AF32C2AF53E6EFC2ADC0D0C0E051
:10042000C0F0D2D3D2AFA8FBA9FCC2D830710281F0
:100430007C53DACF207E0343DA10307E0343DA2088
:10044000D271E580307E01F420E70281538826894D
:1004500027C1B853DACF207E0343DA20307E03432E
:10046000DA10C2D8C271307402C1A47800E58030BD
:0F0470007E01F430E702C1A48859C18B53DACF63
:10047F00207E0343DA20307E0343DA10C2712061FD
:10048F0002A14C53DACF207E0343DA10307E0343B0
:10049F00DA20C2D8D27188548955C3E89552F8E949
:1004AF009553F9E4FB7E027A00C3E8948CE994003B
:1004BF005005755800A13CC3E894C8E99400500852
:1004CF00E4D2E4FB7A0AA119C3E89468E9940150D5
:1004DF0008E4D2E3FB7A0FA119C3E894D0E99402A0
:1004EF005008E4D2E2FB7A1EA119C3E894A0E99464
:1004FF00055008E4D2E1FB7A3CA119C3E89498E9CE
:10050F0094085008E4D2E0FB7A787E00C3E8955651
:10051F00FCE99557FD30E708ECF42401FCEDF4FD00
:10052F00755800C3EC9AED9E500375580188568993
:10053F0057A854A955885289537802C18BC3E8959F
:10054F0026F8E99527F9307C02C16F307B02C16F25
:10055F00307A02C168207502A16FE9FDE8FCA18E17
:10056F00E9C313F9E813F8307902C168E9C313F945
:10057F00E813F8307802C168E9C313FDE813FC20D3
:10058F006126C3EC941CED94024002A1A5ED7018F6
:10059F00C3EC94C850120528C3E528940A5002C131
:1005AF00A4755900D270C1A4E52860021528740003
:1005BF00207F0B7888E67896B40302789EE624FABB
:1005CF00FEE43400FFC3EC9EFCED9FFD920878889B
:1005DF00E6B40327A2085009207D20C2AFD27DA127
:1005EF00F7307D17C2AFC27DC292C291C290C29541
:1005FF00C294C293206902D26BD2AFA2085017E601
:10060F00B4030DECF42401FCEDF43400FD020625D7
:10061F0078007900C16F7888E6B40315EC33FCEDF0
:10062F0033FDC3EC940AFCED9400FD50047C007D77
:10063F0000C3EC94FFED9400400678FF7900C16F82
:10064F00EC856FF0A4C5F0A2F733F87900400302F0
:10065F00068B78FF790002068BE9C313F9E813F8CC
:10066F00307C0EE9600278FFC3E81338F8E43400F9
:10067F00F9C3E894FFE99400400278FF8859D270DB
:10068F00206102C1A4741FF4552F4BF52FC274E4DF
:10069F002B7002D27475291830740375290A3061D2
:1006AF0002C1B820740353DAFE752A06307403753D
:1006BF002A0AD0F0D0E0D0D0C2D3D2AD43E6103268
:1006CF0079010206ED79030206ED790A0206ED794A
:1006DF001E0206ED79640206ED79C80206ED781761
:1006EF00E4D5E0FDD8FAD9F6227A147B7802071404
:1006FF007A107B8C0207147A0D7BB40207147A0BE5
:10070F007BC8020714AC257525017902B27DE4C2BE
:10071F0094D5E0FDE5256002D291D5E0FDC291D5DB
:10072F00E0FDD294D5E0FDE525600A207D02D2924E
:10073F00307D02D290E570D5E0FD207D02C292306F
:10074F007D02C2907496D5E0FDD9C1EAF8D5E0FDDF
:10075F00D8FBDBB1C2948C2522C37C007D0075F0E1
:10076F000005F0EA33FAEB33FB50F6EB13FBEA1319
:10077F00FAC3E9FFE8FEE89AF8E99BF95004EFF9AC
:10078F00EEF8B3EC33FCED33FDD5F0DFEDF9ECF81B
:10079F0022E889F08A20D2D4F8A9F07B0030F70B39
:1007AF007BFFF42401F8E9F43400F9E88520F0A484
:1007BF00ADF0F8E98520F0A4AFF0FEED2EF974004E
:1007CF003FFA7C04C3EA13FAE913F9E813F8DCF4EF
:1007DF008BF030F70AE8F42401F8E9F43400F9E873
:1007EF0089F0C2D4F8A9F02222E547603BC3E53B6C
:1007FF0013F9E53A13F8C3E53E98F8E53F99F95038
:10080F000CC3E89480E994FF4016020833C3E894C0
:10081F007FE994005003020833787F790002083390
:10082F00788079FF8843894422E5476058E543255E
:10083F0040F8E5443541F9854420E4300701F435AB
:10084F0042FA30E709C3EA94F04015020875C3EA8B
:10085F00940F500302087578FF79FF7A0F0208751D
:0F086F00780079007AF0C3E524955E5006E52401
:10087E006009018EE54420E70D018EE54430E70660
:10088E00884089418A4222E54770030208F978A11F
:10089E00E6FAC3E54333F8E54433F91207A0E9302D
:1008AE00E70BC3E89480E994FF401301D0C3E894AA
:1008BE007FE99400500201D0787F790001D07880D2
:1008CE0079FFE820E715C3E52398F84009C3E894BB
:1008DE000140030208F778010208F7E8F424012525
:1008EE0023F840030208F778FF884522E547700396
:1008FE0002095C78A2E6FAA841A9421207A0E930E3
:10090E00E70CC3E89401E994FF4016020933C3E8EB
:10091E0094FFE99400500302093378FF790002092D
:10092E0033780179FFE920E715C3E54598F84009CA
:10093E00C3E89401400302095A780002095AE8F408
:10094E0024012545F8400302095A78FF88242278AD
:10095E00FFC264E52D5406702FD264C3E53B940AA2
:10096E004009C3E52594405002C264E53B6019740A
:10097E00FF853BF0848537F0A4F8C5F0600278FF60
:10098E00C3E895615002A861886022020A36788316
:10099E00E6F520120E6075E8901206CF75E890E528
:1009AE00E820ECFBA8BDA9BE120EF6756B55756C52
:1009BE0000C3740013FD745513FC74552CFC7400A5
:1009CE003DFDECFAEDFBC3E89AE99B4014E56B2480
:1009DE0055F56BE56C3400F56CEA2CFAEB3DFB80BB
:1009EE00E5AE6BAF6CC3E56C13F9E56B13F8C3E9B9
:1009FE0013F9E813F8E56B28F569E56C39F56A7AB1
:100A0E0003C3E913F9E813F8DAF7AA201A70097587
:100A1E006B00756C00020A361AEA6008EE28FEEFCB
:100A2E0039FFDAF88E6B8F6C2275E890227883E6A8
:100A3E00FFE5E820ECF7A8BDA9BE056DC3E56D94F2
:100A4E00084052756D00E9FA79A0E76044EA700734
:100A5E00E56E601B020A71C3E8956E6010E56E507C
:100A6E0006600C14020A7D0460F9020A7DE56EF53B
:100A7E006EC3946D401B755EC0C394044013755EC7
:100A8E0080C39404400B755E40C394044003755EAE
:100A9E000075BB0622E55EF46002055EE56DB407E7
:100AAE000375BB1022743279A387F0A4C5F0A2F7A8
:100ABE0033F8C3E8955E4002A85E88228824882514
:100ACE00886122753A00753B7F2275C820A8CCA993
:100ADE00CD75C824AA38AB3988388939C3E89AF855
:100AEE00E99BF9AA3AAB3BAC3AAD3B7E047F02C31D
:100AFE00EB940440021E1FC3EB940840021E1FC35A
:100B0E00ED13FDEC13FCDEF7C3EA9CFAEB9DFBEF55
:100B1E006009C3E913F9E813F8DFF7EA28FAEB39AD
:100B2E00FB8A3A8B3B400122753AFF753BFF223020
:100B3E006002613D854C50854D51D26043E6802266
:100B4E007892E6FFC3E535948240010FC3E53594F4
:100B5E00A040010FC3EF940640027F057E021E30B7
:100B6E0072010EC3E53B940350060E0E3072010E59
:100B7E00C3E53B940250060E0E3072010EA93BA83F
:100B8E003A7A04C3E913F9E813F8DAF7C3E89EF8E2
:100B9E00E99400F94009C3E89402E99400500478FE
:100BAE0002E4F9E9FBE8FAC3E913FDE813FC884C0B
:100BBE00894DC3EF94036037EF20E00DE82CF8E980
:100BCE003DF9ECFAEDFB020BEAE828F8E939F9C336
:100BDE00E89402F8E99400F97A02E4FBC3EF940377
:100BEE00400D8A4E8B4F884889498C4A8D4B2288FE
:100BFE004E894F8A488B498C4A8D4B223060028138
:100C0E000AD26043E680E52D54066027A83AA93B38
:100C1E00E53494085006E820E002A94D759100C312
:100C2E00E498F594E499F595759104D26053917F0B
:100C3E0043E68022D265753D00752000020C55D228
:100C4E0065753D00752040E52D54066002C265D2E3
:100C5E00AF206005E53D60012278017A02C3E53BD5
:0F0C6E00940540027802C3E53B940A40027803E4
:100C7D00C3E53B940F40027A03306904781E7A0174
:100C8D00206007E53D6003D2AF22D2AF0000C2AFB6
:100C9D00C3E53BFB940F40027B0FEB043073012344
:100CAD0020620123F93069027982E58BC39940D026
:100CBD00053DEAFBE59BF45440B52004DBF681F1DC
:100CCD002065028155C265759100AE3AAF3BC3E414
:100CDD009EF594E49FF595759104D26053917F43F1
:100CED00E68081553065028155D895D2AF223069A5
:100CFD000B0534206016753400020D1920600D208F
:100D0D00650A206B071581158102150A22A84EA9C7
:100D1D004F75910053917FC3E498F594E499F5953F
:100D2D00759104854850854951D26043E6802278FB
:100D3D00003064053065027801E53575F007A4F9DA
:100D4D00E5F028F5F0E9A2F013A2F113A2F213F5E4
:100D5D0035C394785003753578C3E535953640081D
:100D6D00D266C292C291C290306002A175854A507E
:100D7D00854B51D26043E68022C2AFC295C294C268
:100D8D009330720B9002197432D5E0FD020D9C2048
:100D9D007D02D295307D02D293759F11753C020272
:100DAD000EDBC2AF207D02C290307D02C292307246
:100DBD00179001F6C294207D02C293307D02C29538
:100DCD007432D5E0FD020DD8900159306206E5254B
:100DDD006002D291207D03759F01307D03759F21A7
:100DED00753C03020EDBC2AFC295C294C293307242
:100DFD000B9001D37432D5E0FD020E09207D02D295
:100E0D0093307D02D295207D03759F21307D037532
:100E1D009F01753C04020EDBC2AFC2913072179078
:100E2D0001B0207D02C295307D02C293C29474320E
:100E3D00D5E0FD020E4690014730620EE525600AB1
:100E4D00207D02D292307D02D290759F11753C05A6
:100E5D00020EDBC2AFC295C294C29330720B9001E9
:100E6D00857432D5E0FD020E76D294207D03759FF8
:100E7D0001307D03759F21753C06020EDBC2AF204C
:100E8D007D02C292307D02C29030721F90024420CA
:100E9D007D02C295307D02C293207D02C293307DCA
:100EAD0002C2957432D5E0FD020EBB90016B30622B
:100EBD000EE525600A207D02D290307D02D292206F
:100ECD007D03759F21307D03759F01753C01306B4E
:100EDD0013120EF67432D5E0FD7401D5E0FDD295F6
:100EED00D294D293C266D2AF22900145C292C291E2
:100EFD00C290C295C294C293C26222788076FF08D6
:100F0D0076FF0876FF0876FF0876030876040876E4
:100F1D000B087601087601087601788C7601087643
:100F2D00FF0876FF0876FF0876FF0876FF08760340
:100F3D000876FF0876FF0876FF0876250876D00834
:100F4D0076FA0876FA0876040876FF0876010876B0
:100F5D000008767A0876FF087601227887E6FFC2C8
:100F6D00727888E6C394036008C27DE630E102D250
:100F7D007DC27E7889E630E102D27EC3EF940260B5
:100F8D0008758E01D273020F9B758E00C273227885
:100F9D0080E6149000809378A1F67881E614900095
:100FAD00809378A2F6D1F6227886E61490008D9380
:100FBD0078A3F6D1F62222789CE67536FF75370CAC
:100FCD00B402067536A075370AB4030675368275F8
:100FDD00370522227896E6FA7897E6FB307F047A79
:100FED00007BFFC3EB9AFCC3948250027C82756F29
:100FFD0000056FEC856FF0A4C3E5F0948040F222FC
:10100D00D27F120FE11206DE7A007B007C101206F1
:10101D00D4E5592AFA74003BFBDCF37C04C3EB13D3
:10102D00FBEA13FADCF7FEC27F120FE122E5EF2097
:10103D00E6037520000520903FFFE5201460069023
:10104D001DFF1460009304600375EF10C2D353D9D4
:10105D00BF7581C043FF801206CF75EF0043B20309
:0F106D00E5B3240420E702F5B3120EF67580FFF9
:10107C0075A40075F19075D47F75900075A53F75BA
:10108C00F23F75D50075A60175E241120F081215D5
:10109C003C78988670C2AF1206E81206F81206DE8B
:1010AC001206FF1206DE1207061206DE1216501288
:1010BC0006E81206E81206E3C2AFE4F8F6D8FD78AB
:1010CC00C879C8308707D9FBD8F7021C00120F0863
:1010DC0012153C120F68120F9C120FB5120FC3128F
:1010EC000FC4120FE0120FE178988670120EF6758D
:1010FC00885075891275C82475910475D84075A8E7
:10110C002275B80275E690759B80759D0075D10EA1
:10111C0075BC5875BB0675BA1175E8801206CFD22E
:10112C00AF12099943DA01C2D8C2711206E87530C0
:10113C0001D2617B037A0CE55870067A0CDB020154
:10114C00C41206DE20700201C4C270E559C39402B9
:10115C0040E3E52F541F855B5AF55BB55AD7DAD7B8
:10116C00C26153DACF207E0343DA20307E0343DAA8
:10117C0010C2D8C271C2757528001206E33074090A
:10118C00C3E528940A4002D2751206D47802307452
:10119C00027800C3E5599840F0C2AF1206F8120667
:1011AC00F81206F8D2AF1206E87546007888E6B455
:1011BC00030241991206D4788CE6C39401500302C1
:1011CC001299E530C394015003021299207435C36F
:1011DC00E55994FF5003021299C2AF12070DD2AF1A
:1011EC001206E3C3E559940150EFC2AF1206F81290
:1011FC0006D91206F8D2AF1206E3C3E55994FF40A4
:10120C00E90216D57F05D27F120FE11206E3C2AFB9
:10121C00C27F120FE1AE59C3E559947FD2AF40772C
:10122C001206CFC2AF12070DD2AFDFDA110DC3EE2B
:10123C0094057897F61206E812157E1216587F0A56
:10124C00D27F120FE11206E3C2AFC27F120FE1AEE2
:10125C0059C3E559947FD2AF50E41206CFC2AF12F6
:10126C0006F81206D91206F8D2AFDFD4110DEE240F
:10127C00057896F61206E812157E1216871206E30A
:10128C00120FE1C3E55994FF40F30216D5C3E5599B
:10129C00954640038559461206E378017988E7B4F0
:1012AC0003027805C3E55998400221B8C2AF120772
:1012BC000D12070D12070DD2AF1206E8753000E4BF
:1012CC00F531F5320531E531F470390532789AE6AD
:1012DC007819146012783214600D787D14600878D7
:1012EC00FA146003753200C3E53298401715327555
:1012FC0031B478998670C2AF12070DD2AF78988648
:10130C00701206E31206D9E529700530740201C487
:10131C0078012074027806C3E5599840A77888E6CE
:10132C00C3940360031206E3E529700201C4C2AF43
:10133C00120EF6E4F522F523F524F525D2AF7885C7
:10134C008662F53EF53FF540F541F542F56DF54702
:10135C00F52CF52DF535120AD1756D0875BB1012EB
:10136C0006CF120A37E5E820ECFBA8BDA9BEE97050
:10137C0001F8886E120A3B756D0875BB107887E60C
:10138C00FE7602120F687887EEF6C2AF755EFF121A
:10139C000AB385225E85225F852260D2AF75220159
:1013AC00752401752501855D64756501D268D26966
:1013BC00753400120E60120E8A120AD1120AD8125B
:1013CC000B4E0213DD120EF6120F68756D0075BB15
:1013DC0006120C4D120CFB120D1A1207F7120D3CD3
:1013EC00120D86120AD8120B3D120B4E120C0A1259
:1013FC000C42120CFB120D1A1207F812095D120D99
:10140C003C120DAF120AD8120B3D120B4E120C0AE5
:10141C00120C4D120CFB120D1A120838120D3C1244
:10142C000DF3120AD8120B3D120B4E120C0A120CB1
:10143C0042120CFB120D1A120895120D3C120E25BD
:10144C00120AD8120B3D120B4E120C0A120C4D1232
:10145C000CFB120D1A1208FA120D3C120E60120A35
:0D146C00D8120B3D120B4E120C0A120C424E
:10147900120A37120CFB120D1A120A3B120D3C12FA
:101489000E8A120AD8120B3D120B4E120C0A306941
:1014990035206B3285615E85615F855D64756501A7
:1014A90079327A0AC3E53499400FC269D26A8A331C
:1014B900755EFF755FFF0214CFC3E55994014003C0
:1014C9000213DD02150A306A1B206B18E53314700C
:1014D90004C26A61D1F533C3E5599401400302138B
:1014E900DD02150AC3E55C94825016307404E529BF
:1014F900600FC3E53B78F0306B0278609850026169
:10150900DDC2AF120EF67887E6FE7602120F687812
:1015190087EEF6E4F522F523F524F525F562C26890
:10152900D2AF1206CF120EF6307406E52970020109
:10153900C441CB901A0D78201215C0E520B45A0C7D
:10154900A31215C0E520B4A50302155E120F0812F7
:10155900157E02157D901A0378807B0A1215C0A3A7
:1015690008DBF9901A0F788C7B151215C0A308DBDC
:10157900F9901A2422C2AF1215FF1215D9901A0038
:10158900740D1215C5A374021215C5A3741312158F
:10159900C5901A0378807B0A1215C4A308DBF99059
:1015A9001A0F788C7B151215C4A308DBF9121612D1
:1015B9001215F0901A2422E493F622E6438F015380
:1015C9008FFD75EF0275B7A575B7F1F0538FFE2240
:1015D900438F02438F0175EF0275B7A575B7F19077
:1015E9001A0DF0538FFC22901A0D745AB1C5901A36
:1015F9000E74A5B1C5227A3079D07820901A40B1FD
:10160900C0E520F709A3DAF7227A3079D0901A4099
:10161900E7B1C509A3DAF922AB71A872BB01027956
:1016290084BB02027985BB03027986BB04027992E5
:10163900BB05027987BB0602799CBB07027988BB87
:1016490008027989E8F7227C051206E8DCFB22C248
:10165900AF1206F81206FF12070612070D1206D975
:101669001206F81206FF12070612070D1206D91202
:1016790006F81206FF12070612070DD2AF22C2AFF3
:1016890012070D1207061206FF1206F81206D912E2
:10169900070D1207061206FF1206F81206D91207DD
:1016A9000D1207061206FF1206F8D2AF22AE71AF6D
:1016B90072C2AF1206F81206F81206F81206D9DE3F
:1016C900F212070D1206D9DFF8D2AF22D158D15044
:1016D900D150757101757201757300D1B67C05AD74
:1016E900591206E8C3ED955970F5C3E559940140BF
:1016F9000AC3E55994FF4032021711D121B17ED1B5
:1017090058C2AF75EF10D150DCD50573C3E573949A
:1017190003500280C6D1500572E5711490009A9366
:10172900F808C3E57298500280AED150D1500571C6
:10173900C3E57194095002809C120F08B17EC2AFB3
:0517490075EF10D15006
:101A00000D0213FFFFFFFF03040B0101015AA501A3
:101A1000FFFFFFFFFF03FFFFFF25D0FAFA04FF01DE
:051A2000007AFF01FF48
:101A400023585037412320202020202020202020F0
:101A500023424C48454C4923463333302320202031
:101A60002020202020202020202020202020202076
:101C0000C2AFC2D353D9BF7581C043B20343FF8073
:101C1000752438752503B1BF75EF0275E24043F1B5
:101C20008053A47FD287780379E67C1075220075F3
:101C30002300901DCC7B0675249875250130870202
:101C4000813D208708D8FBD9F9DCF781AD308708C2
:101C5000D8FBD9F9DCF781ADB17FE493A3C39A60D7
:101C6000028126DBDDB171600281267B08E493FAF4
:101C7000A3B152DBF87A30B152752200752300B15E
:101C800071EAFCEBFDC3ED94FE400EB1718A278B27
:101C900028ED30E0048A828B83B1717AC270D8C398
:101CA000ED94FE601050CEBD0022EC600675200061
:101CB0000200008100A827A9280809D804D90281B8
:101CC000C9B175EA89AAF281BB0D8199C3ED94036C
:101CD0005049EDA2E092007AC5C3E5829400E58305
:101CE000941C5093200010438F02438F0175B7A5B9
:101CF00075B7F1F030001FA827A9280809438F0104
:101D0000538FFDD804D902A11689AAE275B7A5752B
:101D1000B7F1F0A3A103538FFC81757AC1BD030C09
:101D2000E493A3FAB136DCF8B12E81758177AA224B
:101D3000AB23B152EBFAEA6222752608C3E52313FE
:101D4000F523E52213F52250066323A0632201D573
:101D500026EAB1BFB1BF75260AEAF4200102D28794
:101D6000300102C287B1BFC3134002C201D526EBC6
:101D700022B175EAFB208702A175308702A17A752E
:101D80002608AE24AF25C3EF13FFEE13FEB1C3B197
:101D9000BFC3EA133087024480FA30E703632201AD
:101DA000C3E52313F523E52213F52250066323A090
:101DB000632201D526D9E52265236523F52222AECB
:101DC00024AF250E0FDEFEDFFCD20122424C486517
:0A1DD0006C6934373132F33006013C
:00000001FF
